S31508000000400C0020650100088B0100088D010008DE
S3150800001000000000000000000000000000000000D2
S315080000200000000000000000000000008F0100082A
S315080000300000000000000000910100089D13000860
S31508000040950100089501000895010008950100082A
S31508000050950100089501000895010008950100081A
S31508000060950100089501000895010008950100080A
S3150800007095010008950100089501000895010008FA
S315080000809501000895010008000000009501000888
S3150800009095010008950100089501000895010008DA
S315080000A095010008950100089501000895010008CA
S315080000B095010008000000009501000800000000F6
S315080000C000F002F800F03EF80CA030C808382418F2
S315080000D02D18A246671EAB4654465D46AC4201D172
S315080000E000F030F87E460F3E0FCCB6460126334266
S315080000F000D0FB1AA246AB4633431847F018000057
S3150800010010190000103A02D378C878C1FAD85207F5
S3150800011001D330C830C101D504680C6070470000AF
S315080001200023002400250026103A01D378C1FBD805
S31508000130520700D330C100D50B6070471FB51FBDED
S3150800014010B510BD00F009F91146FFF7F7FF01F0E9
S31508000150E7FB00F021F903B4FFF7F2FF03BC00F058
S3150800016027F900000F4880F308880F480168090E30
S315080001700E4A914205D10E480E4901600E480F49B4
S3150800018001600F4880470F480047FEE7FEE7FEE795
S31508000190FEE7FEE7FEE700000B480C490C4A0D4B4C
S315080001A070470000400C0020040000001F000000FB
S315080001B01810024001000000000001400000000085
S315080001C051140008C100000840060020400C002019
S315080001D0400800204008002010B5202A04DB084605
S315080001E0203AD040002110BD0B462024D340D040F1
S315080001F0A21A91400843194610BD002203098B42F2
S315080002002CD3030A8B4211D300239C464EE00346A7
S315080002100B433CD4002243088B4231D303098B425B
S315080002201CD3030A8B4201D394463FE0C3098B4291
S3150800023001D3CB01C01A524183098B4201D38B01EA
S31508000240C01A524143098B4201D34B01C01A52418D
S3150800025003098B4201D30B01C01A5241C3088B42D2
S3150800026001D3CB00C01A524183088B4201D38B00BD
S31508000270C01A524143088B4201D34B00C01A52415F
S31508000280411A00D201465241104670475DE0CA0F36
S3150800029000D04942031000D34042534000229C46F6
S315080002A003098B422DD3030A8B4212D3FC22890100
S315080002B012BA030A8B420CD3890192118B4208D3D6
S315080002C0890192118B4204D389013AD0921100E038
S315080002D08909C3098B4201D3CB01C01A524183094C
S315080002E08B4201D38B01C01A524143098B4201D379
S315080002F04B01C01A524103098B4201D30B01C01AA4
S315080003005241C3088B4201D3CB00C01A524183081D
S315080003108B4201D38B00C01A5241D9D243088B4273
S3150800032001D34B00C01A5241411A00D20146634616
S3150800033052415B10104601D34042002B00D549427A
S31508000340704763465B1000D3404201B50020C046A3
S31508000350C04602BD704770477047754600F024F8DE
S31508000360AE46050069465346C008C000854618B023
S3150800037020B5FFF711FF60BC00274908B6460026DE
S31508000380C0C5C0C5C0C5C0C5C0C5C0C5C0C5C0C537
S31508000390403D49008D46704710B50446C046C046E4
S315080003A02046FFF7D8FE10BD00487047E00500203C
S315080003B001491820ABBEFEE726000200704700F090
S315080003C0BAF8FCE710B500F081F8012810D0094CFE
S315080003D0207801280CD101F069F8A26861688918AB
S315080003E0FF31F531884203D30020207000F0C4F8AD
S315080003F010BD0000CC00002010B50449012008708B
S3150800040000F006F8FFF7DEFF10BD0000CC00002064
S3150800041010B5044C2078012802D101F047F8A060F5
S3150800042010BD0000CC00002010B500F08CF800F0DC
S3150800043079F801F043F800F0ADFE00F03BF8FFF75D
S31508000440DBFF10BD10B500F076F801F051F800F0AA
S3150800045047F8FFF7B7FF10BD704700000948007856
S31508000460002807D0012807D0022807D0032807D07C
S315080004704020704740207047002070470020704792
S3150800048000207047D800002009480078002807D0C7
S31508000490012807D0022807D0032807D04020704734
S315080004A040207047002070470020704700207047A2
S315080004B0D800002010B501F087F900F0C5FE024902
S315080004C00020087010BD0000D800002010B50024D8
S315080004D001F088F9002800D00124204610BD00004C
S315080004E008B56946064800F0D7FE012807D1054930
S315080004F00020087068460178014801F07DF908BDBA
S3150800050008010020D800002010B5054A1278002AF4
S3150800051002D1C9B200F014FF01F0D8F910BD0000ED
S31508000520D800002010B500F001F810BD10B5642001
S3150800053000F0D8FD10BD10B500F001F810BD10B5DB
S3150800054000F0D6FD10BD10B500F001F810BD72B66A
S31508000550704762B6704770B505460C46164605E004
S3150800056020782870641C6D1CFFF7E5FF3046761E60
S31508000570B6B20028F4D170BD38B500F00FFE0028D9
S3150800058025D000F029F8002821D0FFF765FF00F0F4
S31508000590A9FF00F0A7FA01210D4882690A43826182
S315080005A080690840009000F0F1FD01460120C02254
S315080005B04007FFF7D0FF032006490A688243024333
S315080005C00A6000F0E3FD4468FFF7C3FFA04738BDA3
S315080005D0001002400000014010B501200921C9069B
S315080005E00969884304D00020002803D0002010BDE4
S315080005F00120F9E700F06EFD012010BD0649002034
S31508000600C861064801690422114301610169402253
S315080006101143016170470000E800002000200240F5
S31508000620064A0021D16106490A6902231A430A616A
S31508000630486108694022104308617047E8000020B5
S315080006400020024010B5054B0022DA61044A1369FE
S31508000650012423431361018010BD0000E800002037
S315080006600020024010B500200A4AD168CB060A4984
S3150800067004D5C86902231843C8611020D3685B07EC
S3150800068005D5CB6901242343CB6104210843D060F7
S3150800069010BD000000200240E800002070B50446A6
S315080006A000F0E2FA0546104E0AE0601C08D0002C5D
S315080006B004D000F0D9FA401BA04201D9032070BD2E
S315080006C0F068C007F1D1F068800601D52020F060F7
S315080006D0F068C00602D4F068400703D5FFF7C2FFEA
S315080006E0012070BD002070BD00200240FEB5044602
S315080006F00D4616461F46680A400200902068401CB0
S3150800070005D12046009900F015F900282CD021685B
S315080007100098814206D02046009900F01DF904464B
S31508000720002C23D02068281A05192D1D0098FF30A3
S31508000730FF3002300190FFF7FEFE281B0121001F43
S315080007404902884207D32046019900F005F9044674
S31508000750002C0DD0251D3078761C28706D1C7F1E48
S31508000760002FE8D10120FEBD0020FEBD0020FEBD01
S315080007700020FEBD10B50C480068401C04D00A488D
S3150800078000F05EF900280AD008480068401C04D02A
S31508000790064800F055F9002803D0012010BD0020B6
S315080007A010BD002010BD0000980300209401002011
S315080007B070B505460C460D48411B601E814201D2A4
S315080007C0002070BD284600F053F806462819401E3A
S315080007D000F04EF80146FF2E05D0FF2903D030461B
S315080007E000F006F870BD002070BD0000FFFF00088D
S315080007F0F0B585B00C46012500210391A04200D929
S315080008000025042801D3102C00D90025012D2CD150
S3150800081000F04CF80746204600F048F80646204601
S3150800082000F05EF83018401EC01B401C8001060C04
S315080008300020009001970120029000F001FA0024A0
S31508000840AF020EE0FFF777FE03A9684600F05CF9F1
S31508000850002801D0002506E00198C0190190641C03
S31508000860A4B2B442EED300F09FF9284605B0F0BD15
S3150800087070B5054600240C4EFFF75DFE21460C2098
S3150800088041437058A84209D8891949684018A842AE
S3150800089004D90C204443A019007A70BD641CE4B244
S315080008A00D2CE9D3FF2070BD5019000870B5064617
S315080008B000240A4DFFF73FFE0C2060434019007ADA
S315080008C0B04203D10C204443285970BD641CE4B2DD
S315080008D00D2CEFD30020C04370BD0000501900084E
S315080008E070B5064600240A4DFFF725FE0C20604326
S315080008F04019007AB04204D10C204443601940687C
S3150800090070BD641CE4B20D2CEED3002070BD00004F
S3150800091050190008004870470020000800200349C5
S31508000920C04308600249086070470000940100202F
S315080009309803002010B5CA0501D0002010BD026832
S315080009408A4201D1012010BD02C001225202FFF7DE
S3150800095002FE012010BD000070B504460D460E4883
S31508000960844201D10D4C0AE00D48854202D10A4C59
S31508000970054604E0204600F063F8002807D029461B
S315080009802046FFF7D7FF002803D0204670BD002079
S3150800099070BD002070BD000098030020940100205F
S315080009A0002000080B4801684268511882685118EF
S315080009B0C26851180269511842695118806940186D
S315080009C00449C03109680818002801D0002070477A
S315080009D0012070470020000870B504460D461646EB
S315080009E01348011B681E814201D2002070BD2046B3
S315080009F0FFF73EFFFF2811D06019401EFFF738FFAA
S31508000A00FF280BD0600A40020A49884208D12B46C3
S31508000A10324621460848FFF769FE70BD002070BDC2
S31508000A202B46324621460548FFF760FE70BD00009A
S31508000A30FFFF00080020000898030020940100200A
S31508000A40F8B50646012000903068FFF711FFFF2829
S31508000A5014D000F0F5F800243168A0000F188019AA
S31508000A604568FFF768FD2A4600233946022000F04C
S31508000A70A5F8002804D0002000900AE00020F8BD60
S31508000A803868A84202D00020009002E0641C802C3E
S31508000A90E2D300F089F80098F8BD000008B50020F8
S31508000AA000900E480168491C15D0416882685118A3
S31508000AB0C268511802695118426951188269511859
S31508000AC0C0694018C043401C00906A460421044887
S31508000AD0FFF782FF08BD012008BD0000980300202B
S31508000AE0C020000810B500210648C943016100224C
S31508000AF00261C160C2608162826200F0DBF8002098
S31508000B0010BD000000100240F8B505460F46012644
S31508000B102248017E01290BD0012101762868204C44
S31508000B20012807D02046FFF7B9FD002813D030E08A
S31508000B300220F8BD2046FFF7B1FD002829D1FFF7AE
S31508000B405DFD2046FFF7AAFD064616480169042200
S31508000B50914301611DE00020C04338606C6812E0D3
S31508000B602046FFF75DFD0E48FFF798FD06460D483F
S31508000B700169022291430161300001D03C6008E01E
S31508000B80012080022418A868696880024018A042DB
S31508000B90E6D80248002101763046F8BDE800002074
S31508000BA050C3000000200240034801698022114317
S31508000BB0016100207047000000200240F0B51FB414
S31508000BC0074615461E4600241A48017E012907D005
S31508000BD0012101761848FFF761FD002803D025E0BA
S31508000BE0022005B0F0BD012F03D0022F03D0042741
S31508000BF01AE0012718E0022716E0220128463146A6
S31508000C00FFF7EAFA81B2019862001018FFF71AFD99
S31508000C100948FFF743FD09490A69520852000A6163
S31508000C20002803D1641CE4B2BC42E6D30149002281
S31508000C300A76D6E7E800002050C3000000200240EC
S31508000C40002006490A69120607D5054A4A60054A78
S31508000C504A600969090600D501207047002002404C
S31508000C6023016745AB89EFCD00B500F01FFC00BD39
S31508000C7010B506480168102211430160002000F0F3
S31508000C8007F800F03BF8002010BD000000200240E5
S31508000C9010B5044600F07AF87D21C900FFF7ADFAD1
S31508000CA000F07AF800222146501E00F06BF800206A
S31508000CB010BD000010B500F045F9FF2101310D48BF
S31508000CC0816200F0A3F80920C00600F09FF8012110
S31508000CD049040948C2698A43C2618A004369934341
S31508000CE0436142698A4342618169490849008161D1
S31508000CF010BD00000008004800100240F0B587B09B
S31508000D0001201E4CA1690143A161A069C007C00F5B
S31508000D10009001256D04284600F05CF8A80000F054
S31508000D2059F8E1692943E161E06928400090A7156F
S31508000D300197012502950024039404940594104E06
S31508000D4001A9304600F0AAF8B76201950294059405
S31508000D500926F60601A9304600F0A0F80C200190F5
S31508000D60022002900320039004940594069501A995
S31508000D70304600F093F807B0F0BD000000100240BE
S31508000D800008004810B500F0D1F910BD0148006808
S31508000D9070470000C000002010B50949401E88426F
S31508000DA001D9012010BD074C60610321081F00F01E
S31508000DB0BDF90020A06107202061002010BD0000B9
S31508000DC0FFFFFF0000E000E010B5FFF751FF00F05D
S31508000DD0E7FA10BD08B504494A6902434A614969F8
S31508000DE00140009108BD00000010024002498A6ACD
S31508000DF002438A62704700000010024002498A6A6C
S31508000E0082438A62704700000010024070B50124D0
S31508000E100921C906884207D165042846FFF7E6FF77
S31508000E202846FFF7EBFF2EE01849884207D105024E
S31508000E302846FFF7DBFF2846FFF7E0FF23E01449C3
S31508000E40884207D105022846FFF7D0FF2846FFF754
S31508000E50D5FF18E00F49884208D101252D052846F7
S31508000E60FFF7C4FF2846FFF7C9FF0CE00A49884286
S31508000E7008D10125AD052846FFF7B8FF2846FFF734
S31508000E80BDFF00E00024204670BD000000040048B5
S31508000E9000080048000C004800140048F0B500237C
S31508000EA03EE001249C402240002A38D04F68144670
S31508000EB00668644365006519AE4367433E430660AA
S31508000EC04E68012E01D0022E05D18F6886686743C9
S31508000ED0AE433E4386600F69C668AE4325467D43EA
S31508000EE02E43C6604D68022D19D1FF2A0AD84D69CE
S31508000EF0066A544354432201121B96436C43264305
S31508000F0006620CE04D69140A224662436243624354
S31508000F101401A61A446A6A43B443144344625B1C28
S31508000F200A681446DC40BCD14A68012A01D0022A64
S31508000F3006D10A68C968436893434A431343436022
S31508000F400120F0BD10B51548016801221143016062
S31508000F500168F822914380231943016010494160D2
S31508000F60104901600168DC02A1430160002141606B
S31508000F70446B94431C434463426B520852004263D9
S31508000F80426B04239A434263C1620163BF2212047F
S31508000F908368134383608160012010BD00100240FE
S31508000FA00CF8FFF0FFFFF6FE10B5044600F01AF93C
S31508000FB0206000F0FBF8606000F006F9A06010BD44
S31508000FC010B50146002000290FD1114A116B890777
S31508000FD0890F01290AD0022912D0032909D000F065
S31508000FE001F900F0E3F800F0EFF810BD00F0FAF8A8
S31508000FF010BD11688907C90F0029F9D0054810BD29
S31508001000116A8907C90F0029F9D00120C00310BD4C
S315080010100010024000127A0001490860704700007B
S31508001020C0000020FEB504460D46002600202168B3
S31508001030C907C90F002942D1EA686968AB69114333
S315080010402A691A43114322681E4B1A40114321602C
S31508001050A968626803231B039A430A4362606969A5
S31508001060A2681B119A430A43A26017498C4202D10F
S31508001070FFF7A6FF06E015498C4203D16846FFF73D
S3150800108093FF029800281AD02968002917D001264C
S31508001090AA69F3039A420CD140004A088018FFF760
S315080010A0ACF880B20A4901400007420F0A43E260E1
S315080010B005E04A081018FFF7A0F880B2E06030464D
S315080010C0FEBD0000F369FFFF003801400044004000
S315080010D0F0FF0000FF2001300149886270470000D8
S315080010E0000800480149488070470000C4000020F5
S315080010F010B500F0DBF90B4C616888420DD32278F5
S31508001100FF2001300849002A08D000222270886290
S3150800111000F0CCF961884018606010BD0122227089
S315080011208861F5E7C4000020000800488307FF220D
S31508001130DB0E9A408907090E994000280BDA00074A
S31508001140000F0838830808489B001818C36993439A
S315080011500B43C3617047830804489B00181803684B
S3150800116093430B430360704700ED00E000E400E0A2
S3150800117010B5FFF793FC002802D0FFF7FBFA10BD65
S31508001180002010BD10B5FFF713FB10BD10B5FFF713
S31508001190C1FB10BD10B5FFF7C1FB10BD10B5FFF7B9
S315080011A001FC10BD10B5FFF717FC10BD04494968CE
S315080011B0F0221140034A0909515CC84070470000F3
S315080011C0001002402E190008044949680722120235
S315080011D01140034A090A515CC84070470010024092
S315080011E03E19000810B5074841680C20014006481A
S315080011F0002905D0042903D0082901D100F006F8F2
S3150800120010BD00000010024000127A0010B50C4C08
S3150800121061680122120411400A48002902D091424D
S3150800122000D14000E16A0907090F491CFEF7E5FFEE
S3150800123061680F2292041140890C891C484310BD2D
S315080012400010024000093D0010B588B0E1200002F8
S31508001250019000200290039004900C2105910690BD
S315080012600790054C01A92046FFF7DCFE21680122FC
S315080012701143216008B010BD00440040024600201A
S315080012800449CB699B06DB0F002B02D0888C1070B3
S315080012900120704700440040F3B581B00F461B4C4F
S315080012A0002560781A4E00280FD020783018401C88
S315080012B0FFF7E4FF012818D000F0F8F861686431F8
S315080012C0884200D965700020FEBD1148FFF7D6FF99
S315080012D00128F8D13078401E3F28F4D800F0E6F807
S315080012E06060257001206070EDE72078401CC2B26E
S315080012F0227030789042E6D1711C0198FFF72BF9DD
S315080013006570207838700120FEBD0000E0000020DE
S315080013109C05002070B5094D288500F0C7F80446DD
S315080013200A3405E0FFF707F900F0C0F8A04204D830
S31508001330E8690006C10F0029F4D070BD00440040DA
S3150800134070B506460D46402D03D9812108A0FFF742
S3150800135036F82846FFF7DEFF002406E0FFF7EBF82D
S31508001360305DFFF7D7FF641CA4B2AC42F6D370BD5C
S315080013702E2E5C2E2E5C2E2E5C2E2E5C536F7572D6
S3150800138063655C41524D434D305F53544D3332468D
S31508001390305C72733233322E6300000070470000EF
S315080013A010B50121244802688A430A43026000688E
S315080013B00840002803D16A2120A0FFF700F8224838
S315080013C001680122920411430160016892101143D9
S315080013D0016001688903C90F0029FAD041683D22D6
S315080013E0120491431122120411434160C16A09098A
S315080013F00901C162016801221206114301600168F0
S315080014008901C90F0029FAD04168F0229143416049
S3150800141041680722120291434160022142689208FC
S3150800142092000A4342600C22416811400829FBD108
S315080014300648FFF7F1FD10BD002002402E2E5C6D18
S3150800144061696E2E6300000000100240006CDC0229
S31508001450134801680122114301604168114A11408D
S3150800146041600168104A1140016001680122920436
S315080014709143016041683F22120491434160C16A69
S3150800148009090901C162016BFF22543291430163C4
S31508001490416B49084900416300218160704700009B
S315080014A0001002400CB8FFF8FFFFF6FE00B500F08A
S315080014B01FF80148006800BDDC00002000B500F0F8
S315080014C011F806480449416100218161052202613B
S315080014D00348016000BD00007FBB000000E000E09B
S315080014E0DC000020014900200861704700E000E0A8
S315080014F004480069C00303D503480168491C016014
S315080015007047000000E000E0DC00002010B5084C41
S31508001510FF21E1704168E21DA06C00F043F92071DB
S3150800152000206071A071082120464030818010BDDE
S315080015304801002070B500F0CFF90E4C0125257042
S31508001540FF20E0700021102020716171FEF786FFF0
S31508001550A071FEF799FFE071FEF796FF000A207268
S315080015606572A5722046082140308180FFF712FE79
S3150800157070BD00004801002010B5064C0020207000
S3150800158000F0AAF9FF20E070012120464030818052
S3150800159010BD0000480100200748FF21C170074917
S315080015A0816400210171417181710721C01C41606C
S315080015B008213D30818070474801002046190008FF
S315080015C00648FF21C170002101714278427181717C
S315080015D0C1710172062140308180704748010020A0
S315080015E070B50446FEF73AFF6178801E884203DA32
S315080015F0222000F077F970BD104DFF20E870012118
S31508001600284640308180617800290AD0A21CA86C3F
S31508001610FFF7C8FD00280CD06178A86C4018A864AC
S3150800162070BDFFF7A5FD0028FAD1312000F05AF960
S3150800163070BD312000F056F970BD00004801002049
S3150800164010B5094C4168A06CFFF79CFD002806D030
S31508001650FF20E070012120464030818010BD3120F6
S3150800166000F040F910BD00004801002070B505469D
S31508001670FEF7F4FE0C4C411E6A1CA06CFFF792FDA7
S3150800168000280CD0FF20E070FEF7E8FEA16C401E93
S315080016904018A064012120464030818070BD312069
S315080016A000F020F970BD00004801002010B5312077
S315080016B000F018F910BD000010B5FEF75DFF0449EB
S315080016C0FF20C870024801214030818010BD00000B
S315080016D04801002070B5084CFF20E07000252571F0
S315080016E06571FEF7BBFEA071E5712572657207216B
S315080016F020464030818070BD480100200449FF2201
S31508001700CA70406888640248012140308180704769
S315080017104801002070B50446FEF7A0FE6178401E19
S31508001720884203DA222000F0DDF870BD094D6168B1
S31508001730A9646278281DFEF70EFFFF20E87061781D
S31508001740A86C4018A86460782946401C40318880F7
S3150800175070BD00004801002010B5002000F0C2F856
S3150800176010BD000070B50546FEF778FE6A78401E83
S31508001770904203DA222000F0B5F870BD084C201D0F
S31508001780A16CFEF7E8FEFF20E0706978A06C4018AF
S31508001790A06468782146401C4031888070BD0000EE
S315080017A048010020F8B504460E461746002505E010
S315080017B02078641C4019C5B2FEF7BDFE761E701C63
S315080017C0F6D13D600120F8BD054A002010709064EE
S315080017D011464031C870888090705070704700007C
S315080017E04801002003480078002801D001207047EE
S315080017F0002070474801002070B50178324CFF2957
S315080018000FD02278012A5ED1F42921D013DCD02901
S3150800181036D009DCC92930D0CC293DD0CF293ED1D4
S3150800182037E0FFF787FE3DE0D1292FD0D2292AD00D
S31508001830F32934D112E0F5390B0000F064F80A06F2
S315080018400C303030123015181B30FFF78BFF29E0AB
S31508001850FFF760FF26E0FFF751FF23E0FFF756FE8C
S3150800186020E0FFF799FE1DE0FFF776FF1AE0FFF785
S31508001870A7FE17E0FFF780FE14E0FFF7F7FE11E07A
S31508001880FFF7AEFE0EE0FFF725FF0BE0FFF7D8FEE9
S3150800189008E0FFF711FF05E0FFF708FF02E0202048
S315080018A000F020F8084D4035E878012802D11020CC
S315080018B000F018F80421695E002904DD0120E870AB
S315080018C0E01C00F01BF870BD48010020014800210B
S315080018D0C170704788010020014900204870704790
S315080018E0480100200449FE22CA70087102480221F4
S315080018F040308180704700004801002010B589B249
S31508001900FEF702FE10BD30B47446641E2578641CCA
S31508001910AB4200D21D46635D5B00E31830BC184736
S31508001920FFF752FAFEF780FDFEF78CFDFCE7000094
S315080019300000000000000102030406070809000071
S315080019400000010203044F70656E424C540000000B
S315080019500020000800080000040000000028000815
S31508001960000800000500000000300008000800001C
S315080019700600000000380008000800000700000004
S3150800198000400008000800000800000000480008A1
S3150800199000080000090000000050000800080000C8
S315080019A00A00000000580008000800000B000000AC
S315080019B000600008000800000C000000006800082D
S315080019C0000800000D000000007000080008000074
S315080019D00E00000000780008000800000F00000054
S315080019E00080000800800000100000000C1A0008A3
S315080019F0C00000202800000004010008341A00086E
S31508001A00E8000020580B00002001000800127A00A8
S31508001A1000000000000000000000000000000000B8
S31508001A2000000000040000000000000000000000A4
S30908001A3000000000A4
S705080000C131
